:1017020050543130305838002449643A207363739E
:101712005F313030312E6320343333392032303070
:10172200382D30392D33302031353A32303A353692
:101732005A2072697474405053492E434820240041
:10174200040800000150543130305F300001014084
:10175200040800000150543130305F31000101446F
:10176200040800000150543130305F32000101485A
:10177200040800000150543130305F330001014C45
:10178200040800000150543130305F340001015030
:10179200040800000150543130305F35000101541B
:1017A200040800000150543130305F360001015806
:1017B200040800000150543130305F370001015CF1
:1017C200013400000050545459505F300001016050
:1017D200013400000050545459505F31000101613E
:1017E200013400000050545459505F32000101622C
:1017F200013400000050545459505F33000101631A
:10180200013400000050545459505F340001016407
:10181200013400000050545459505F3500010165F5
:10182200013400000050545459505F3600010166E3
:10183200013400000050545459505F3700010167D1
:101842000000000000000000000000000000000096
:08185200020100030201000382
:0E2859000119010308FF1742010B00010C00DA
:09288F001515A815EFF605152238
:052898008F347F0022D7
:1026F9008B348A358936120CB6AB37AA38A9391208
:102709000CFCAB34AA35A936900001120CCFAB37BB
:0D271900AA38A939900001120D0E7F02228E
:10258F00C2DAE4FEC2D9C2DDD2D90EBE04F6E4FE31
:10259F007C08C2D9EF5CD394004003D38001C3926F
:1025AF00DDD2D9ECC313FC0EBE04E7D2DAC2DAE4F3
:1025BF00FE7C80C2D9ED5CD394004003D38001C36D
:0E25CF0092DDD2D9ECC313FC0EBE08E7D2DABF
:0125DD0022DB
:1025DE00C2A4E4FEC2A3C2A7D2A30EBE04F6E4FEBA
:1025EE007C08C2A3EF5CD394004003D38001C39256
:1025FE00A7D2A3ECC313FC0EBE04E7D2A4C2A4E47C
:10260E00FE7C80C2A3ED5CD394004003D38001C353
:0E261E0092A7D2A3ECC313FC0EBE08E7D2A411
:01262C00228B
:061E58008B428A4389441D
:101E5E00C2DAE4F545C2D9E545B40103D38001C326
:101E6E0092DDD2D90545E545B404EAE4F5457E0890
:101E7E00C2D9EF5ED394004003D38001C392DDD26A
:101E8E00D9EEC313FE0545E545B404E4D2DAC2DA51
:101E9E00E4F545AB42AA43A944120EC60000000069
:101EAE00AB42AA43A944120E237801120E10120E51
:101EBE0043C2D9AB42AA43A944EBC0E0EAC0E0E971
:101ECE00C0E0120E5DA2DCE4334BFFEAFEE9FDE852
:101EDE00FCD0E0F9D0E0FAD0E0FB120E43D2D905E7
:081EEE0045E545B418BAD2DA4B
:011EF60022C9
:061EF7008B428A4389447E
:101EFD00C2A4E4F545C2A3E545B40103D38001C3F3
:101F0D0092A7D2A30545E545B404EAE4F5457E085C
:101F1D00C2A3EF5ED394004003D38001C392A7D236
:101F2D00A3EEC313FE0545E545B404E4D2A4C2A453
:101F3D00E4F545AB42AA43A944120EC600000000C9
:101F4D00AB42AA43A944120E237801120E10120EB1
:101F5D0043C2A3AB42AA43A944EBC0E0EAC0E0E907
:101F6D00C0E0120E5DA2A6E4334BFFEAFEE9FDE8E8
:101F7D00FCD0E0F9D0E0FAD0E0FB120E43D2A3057D
:081F8D0045E545B418BAD2A4E1
:011F95002229
:1013B00030DB030215587B007A00793A7F04121E55
:1013C00058AF3DAE3CAD3BAC3AE4120BF7E4FBFA50
:1013D0007980784B120AED7B0A7AD77923783F120D
:1013E00009E48F418E408D3F8C3E7460250BF58261
:1013F000E43401F583E0B4010A7B6F7A12798378D3
:101400003A8010AF41AE40AD3FAC3E7B0A7AD7790F
:1014100023783C120AED8F418E408D3F8C3E7F75C4
:101420007E787D0C7C35AB41AA40A93FA83E1209CD
:10143000E4AB41AA40A93FA83E1209E4AB41AA404F
:10144000A93FA83E1209E4ECC0E0EDC0E0EEC0E028
:10145000EFC0E07FFA7EED7D6B7C3AAB41AA40A9FC
:101460003FA83E1209E4AB41AA40A93FA83E120999
:10147000E4D0E0FBD0E0FAD0E0F9D0E0F81208F3D5
:10148000ECC0E0EDC0E0EEC0E0EFC0E07F177ED939
:101490007D167C40AB41AA40A93FA83E1209E4D08A
:1014A000E0FBD0E0FAD0E0F9D0E0F81208F37BD30B
:1014B0007A4D79E278411208F38F418E408D3F8C4E
:1014C0003E7B337A93798878431208EF8F418E40C0
:1014D0008D3F8C3EE4FFFE7DC87C42AB41AA40A913
:1014E0003FA83E1209E4E4FBFAF9783F1208F31230
:1014F0001D05E4FBFA79C87842120AED8F418E404F
:101500008D3F8C3EE4FFFE7D487CC2AB41AA40A9E2
:101510003FA83E120B8A500C7541007540C0753FC4
:1015200079753EC4C2AFAF41AE40AD3FAC3EE50BB6
:1015300025E025E02440F582E43401F583120E898C
:10154000D2AFE50B045403F50B90185293C454F03A
:08155000448DFD7F0212258F7E
:011558002270
:1015590030A5030217017B007A00793A7F04121E35
:10156900F7AF3DAE3CAD3BAC3AE4120BF7E4FBFA06
:101579007980784B120AED7B0A7AD77923783F1262
:1015890009E48F418E408D3F8C3E7460250CF582B5
:10159900E43401F583E0B4010A7B6F7A1279837828
:1015A9003A8010AF41AE40AD3FAC3E7B0A7AD77965
:1015B90023783C120AED8F418E408D3F8C3E7F751A
:1015C9007E787D0C7C35AB41AA40A93FA83E120923
:1015D900E4AB41AA40A93FA83E1209E4AB41AA40A5
:1015E900A93FA83E1209E4ECC0E0EDC0E0EEC0E07E
:1015F900EFC0E07FFA7EED7D6B7C3AAB41AA40A952
:101609003FA83E1209E4AB41AA40A93FA83E1209EE
:10161900E4D0E0FBD0E0FAD0E0F9D0E0F81208F32A
:10162900ECC0E0EDC0E0EEC0E0EFC0E07F177ED98E
:101639007D167C40AB41AA40A93FA83E1209E4D0DF
:10164900E0FBD0E0FAD0E0F9D0E0F81208F37BD360
:101659007A4D79E278411208F38F418E408D3F8CA3
:101669003E7B337A93798878431208EF8F418E4015
:101679008D3F8C3EE4FFFE7DC87C42AB41AA40A968
:101689003FA83E1209E4E4FBFAF9783F1208F31285
:101699001D05E4FBFA79C87842120AED8F418E40A4
:1016A9008D3F8C3EE4FFFE7D487CC2AB41AA40A938
:1016B9003FA83E120B8A500C7541007540C0753F1A
:1016C90079753EC4C2AFAF41AE40AD3FAC3EE50C0B
:1016D90025E025E02450F582E43401F583120E89D2
:1016E900D2AFE50C045403F50C90185693C454F08A
:0816F900448DFD7F021225DE85
:0117010022C5
:1020310075840F75A4F175A5AA75A69CE4F5A7F59D
:102041009C759D27F59EF59FEF6013E4FE74602E4D
:10205100F582E43401F5837401F00EBE08EFD2D8A5
:102061007D527F0312258F7D037F0112258FE50BA2
:10207100C454F0448FFD0F12258FD2A27D520F124E
:1020810025DE7D037F011225DEE50CC454F0448F6B
:10209100FD0F1225DEC374FF95B0FDC454F0C45486
:1020A1000F75F00AA4FFAEF0EDC4540F7C00540F7D
:1020B1002F785BF6EC3E18F6E4FECFEECF12288FB8
:0420C1000EBE08F651
:0120C50022F8
:060003001213B0021559B2
:0D286B00245265763A20343637332024009D
:10109C00E47880F6122846D28575840F75E104E455
:1010AC00F5E275E344F58475B7B075840F758A83E2
:1010BC00F597438901758D01758F01758E04F53C8B
:1010CC00F53D053DE53D7002053C640F453C70F275
:1010DC00438902E4F53CF53DAE3CAF3DE4FCFD7BC1
:1010EC00507AC3F9F8D3120DE9400FE58920E40AD0
:1010FC00053DE53D70E2053C80DE7597021227F553
:10110C00E4FF12281443EF04E4F53CF53D7D01AFF8
:10111C003D122726053DE53D7002053CC39401E5D3
:10112C003C940040E8E4F520C20AC208C20EC20D8D
:10113C00C20C7880F608F67853F618F67858F6F55F
:10114C003CF53D7400253DF582E43400F583E4F074
:10115C00053DE53D7002053CB400E8E53CB401E317
:10116C00E4F53CF53D7400253DF582E43401F5834E
:10117C00E4F0053DE53D7002053C6440453C70E5FE
:10118C00E4F584E5EF20E10CE5EF5408D39400403E
:10119C0003D38001C392037D08E4FF1227AAE478ED
:1011AC0057F67850F6AB08AA09A90A7850E6FF75ED
:1011BC00F010A4F58285F083120CCFFE785726F63A
:1011CC00EE600578500680DDEFD394004030AB081C
:1011DC00AA09A90A90000D120EE0120CB6FF745564
:1011EC00120CFC120CB664556002D20C74AA120CD0
:1011FC00FC120CB664AA6002D20CEF120CFCE4F5E3
:10120C0084E5EF5402D3940040047F018002E4FF94
:10121C00121B688F3BE53B20E036C20974FF785AFD
:10122C00F608F608F608F67E007F107D007B007A43
:10123C00007960120F367541FF75421775430275C0
:10124C0044007545107B007A00796012253D8002C0
:10125C00D209902872E493FF3395E0FEEF24D0FF7F
:10126C00EE34FFFE7C007D64120D30AA06AB0790B5
:10127C002871E493FF3395E0FEEF24D0FFEE34FFAA
:10128C00FE7C037DE8120D30EF2BFBEE3AFA902832
:10129C0073E493FF3395E0FEEF24D0FFEE34FFFEB2
:1012AC007C007D0A120D30EF2BFFEE3AFEA3E49387
:1012BC00FD3395E0FCED24D0FDEC34FFCD2F785FB1
:1012CC00F6ED3E18F6E53B30E103021387E4F53CFE
:1012DC00F53DE53DC4F8540FC868FFE53CC454F037
:1012EC0048FEAB08AA09A90A8F82F583120CCF70AD
:1012FC000302137EE92FF9EA3EFA900004120CCF98
:10130C0020E264E4F53AE53AC37819965059E53D84
:10131C00C4F8540FC868FFE53CC454F048AB08AAA5
:10132C0009A90A8F82F583120CCFFF7E00C006C07C
:10133C00077D00E53DC4F8540FC868FFE53CC45474
:10134C00F048FEE92FF9EA3EFA90000D120EE07813
:10135C0057E6853AF0A429F9EA35F0FAD007D00619
:10136C00120F36053A809F053DE53D7002053C02A3
:10137C0012DE7F01122031C20B8007E4FF122031F4
:10138C00D20BE4F53CF53D7A007B967D03AF3D1224
:10139C0020C6053DE53D7002053CC39401E53C9437
:0313AC000040E41A
:0113AF00221B
:05289D007858E6FF225F
:0300230002185A66
:10185A00C0E0C0F0C083C082C0D075D000C000C054
:10186A0001C002C003C004C005C006C00730993ECB
:10187A00C2997853067953E77881667015F67853DA
:01188A00F667
:0D188B0075220A75231300D523FCD522F623
:04189800D285801C59
:0D189C0075221475231300D523FCD522F608
:1018A9007853E62400F582E43401F583E0F59920C4
:1018B9009803021955209A08200A05C2980219515D
:1018C900C29A7852E6062400F582E43400F583E5ED
:1018D90099F0C298E6FFB40112900000E0FE70038F
:1018E900F68069EE540724027859F6EFB4020D78B0
:1018F90059E6B40907900001E02403F67852E6FF9F
:10190900B40007E4B40103F68042EFC37859964066
:101919003B7852E624FFFDE434FFFC7B017A007931
:10192900001221577852E624FFF582E434FFF5834B
:08193900E06F600476008014E9
:0D19410075221475231300D523FCD522F662
:10194E0012002678527600D007D006D005D004D0EB
:10195E0003D002D001D000D0D0D082D083D0F0D02E
:02196E00E03265
:10226F00900001E075F010A4AB08250AF9E50935D7
:10227F00F0FA90000D120EE07858E6FF18E68FF096
:10228F00A42526F582E435F0F583120CCFFF7B00F1
:04229F007A00792424
:1022A3008F348B358A368937E4F584EA494B601CD1
:1022B300AB35AA36A937120CB6FFE534FD7C001204
:0C22C3002878AB35AA36A937EF120CFCC6
:0D22CF0075381475391300D539FCD538F673
:0E22DC008534997F011227533099FDC2992253
:1026C3009001007478F07852E624FFF582E434FF39
:0926D300F583E0900101F07F02A3
:0926DC00E4F5847881EFF6C28573
:0D26E50075341475351300D535FCD534F669
:0726F200900100E0F59922C0
:10267B00C9EFC9E964017028EDC39B40347819E6B2
:10268B00FFEB2FFFE433FEEDC39FEE6480F8748005
:10269B0098501ED20AC3ED9B7858F67854760122D7
:1026AB00B90214ED6B700AD20A7858F67854760298
:0826BB0022C20AE47854F62261
:10242800C9EFC9BAFF15BBFF12ED6B7002EC6A70F9
:1024380049D20A7858F67854E9F622E964017025F9
:10244800C3ED9BEC9A401C7819E62BFFE43AFEC3D7
:10245800ED9FEC9E500DD20AC3ED9B7858F6785448
:102468007601228015B90218ED6B7002EC6A700AC9
:10247800D20A7858F67854760222C20AE47854F6DA
:012488002231
:10002600900000E0FF54F8F525E4F584EF120F1078
:1000360000730900800A009310009C1100AD1200A5
:10004600C41900DA1A00FF20010828018929028B49
:100056003302C63702F539030F41031A4903245008
:10006600036C610255700364980000039C900001C4
:10007600E0FD785BE6FB7F018027900001E0FCA3B2
:10008600E0FD785AE6FA08E6FB7F01802BD20A7873
:1000960054760302039C900001E0FD785DE6FB7F49
:1000A6000212267B02039C900001E0FCA3E0FD788F
:1000B6005CE6FA08E6FB7F0212242802039C900005
:1000C60001E0FD785BE6FB7F0112267B200A030236
:1000D600039C801A900001E0FCA3E0FD785AE6FA42
:1000E60008E6FB7F01122428200A0302039C9001E4
:1000F600007478F07F01020399E4F58475EF10022D
:10010600039CC2ACE4F524C285FB7A0079247F7F88
:100116001222A37B007A0079247F181222A37B0087
:100126007A0079247F051222A37850E612229C7861
:100136005AE612229C785BE612229C785CE6122232
:100146009C785DE612229C785EE612229C785FE639
:1001560012229CE4F52674602526F8E612229C05F8
:1001660026E526C3941040EE7B007A007900AF2482
:030176001222A3AF
:0D01790075320A75331300D533FCD532F60C
:10018600020240900001E0FFC3785096400302024D
:1001960047EF75F010A4250AF9E50935F085082F13
:1001A600F5308931C2ACE4F524C285FB7A007924A6
:1001B6007F7F1222A37B007A0079247F0D1222A36F
:1001C600AB2FAA30A931120CB612229CAB2FAA3043
:1001D600A931900001122299AB2FAA30A9319000C3
:1001E60002122299AB2FAA30A9319000031222994C
:1001F600AB2FAA30A931900004122299E4F526AB60
:100206002FE5312405F9E43530FA7E00E92526F993
:10021600EE3AFA120CB612229C0526E526C394087D
:0D02260040DD7B007A007900AF241222A396
:0D02330075320A75331300D533FCD532F651
:10024000D285D2AC02039C9001007478F0E4A3F054
:100250007F020203991228337870120E7D900100FC
:10026000747CF07870E6A3F008E6A3F008E6A3F04B
:1002700008E6A3F07C007D057B017A01790012215C
:1002800057900105EFF07F06020399900001E0FF0F
:10029000B4010FA3E0FDA3E0785ACDF608EDF60215
:1002A0000364EFB4020A900002E0785AF602036495
:1002B000900001E0B4030CA3E0FFA3E0785CCFF66C
:1002C00008EFF6020364E4F526900001E0FFE5265E
:1002D000C39F501B74022526F582E43400F583E0A9
:1002E000FF74602526F8EFF60526E526B410DAE45B
:1002F000786FF6806F7A007B327D017858E6FF12C6
:1003000020C6900001E0FDE4FF1227AA02039C90A2
:100310000001E024FF920202039C900001E024FF10
:10032000920180787858E66005752802800B200DD0
:100330000575280380037528019001007479F0A3E6
:10034000E528F07C007D027B017A017900122157BB
:10035000900102EFF07F031226DCE5286401703C77
:10036000D20E8002D208788076F180307A007B321B
:100370007D017F001220C69001007479F090000189
:10038000E0900101F07C007D027B017A017900128E
:100390002157900102EFF07F031226DCE52564A0CF
:1003A00060030205AB900000E064A1600302049BBF
:1003B000A3E0C37850964003020490AB08AA09A9B1
:1003C0000AE0FF75F010A4F58285F083120CCFF5DA
:1003D00028EF75F010A429F9EA35F0FA900004121C
:1003E0000CCF30E237900001E01228988F2890015E
:1003F00000747FF0A3E528F02402FDE433FC7B01C8
:100400007A01790012215774022528F582E434011B
:10041000F583EFF0E5282403FF0205A8900001E032
:10042000FF122898C2ACE4F524C285E528D39406CF
:10043000402B7B007A0079247F7F1222A37B007AF5
:10044000007924AF281222A3E4F526E526C39528D7
:10045000500712226F052680F205288018E528240F
:100460007812229CE4F526E526C39528500712222F
:100470006F052680F27B007A007900AF241222A358
:0D04800075320A75331300D533FCD532F602
:10048D0002059A9001007478F07F010205A8900092
:10049D0000E064A260030205AB7850E6FFA3E0FE26
:1004AD00C39F40030205A0A3E0FDC39F40030205C7
:1004BD00A0EE9D40030205A0900001E0F526E4F5B5
:1004CD002DF52E900002E0FFE526D39F5026AF2696
:1004DD00122898AB08AA09A90A75F010E526A4F50B
:1004ED008285F083120CCF252EF52EE4352DF52DBA
:1004FD00052680CFC2ACE4F524C285FB7A007924B1
:10050D007F7F1222A3C3E52E9480E52D9400500227
:10051D008007E52D448012229CAF2E12229D900063
:10052D0001E0F526900002E0FFE526D39F5046E45A
:10053D00F527AB08AA09A90A75F010E526A4F582DE
:10054D0085F083120CCFFFE527C39F5024E5267558
:10055D00F010A429F9EA35F0FA90000D120EE078AA
:10056D0058E6FF18E68FF0A4252712229205278062
:10057D00C1052680AF7B007A007900AF241222A33B
:0D058D0075320A75331300D533FCD532F6F4
:10059A00D285D2AC800B9001007478F07F011226CC
:1005AA00DCE5256458704DFA7B327D017858E6FF08
:1005BA001220C67537017538017539017B017A0039
:1005CA0079011226F98F28E5282478900100F0EFA6
:1005DA002401FDE433FC7B017A017900122157746E
:1005EA00012528F582E43401F583EFF0E528240299
:1005FA00FF1226DCE52564806009E525648860032E
:10060A000207B37854E6B4010F7A007B327D017891
:10061A0058E6FF1220C6801AE4F526E526C37819A3
:10062A0096500F7A007B327D01AF261220C605262E
:10063A0080E9900000E05407F528B4070A752701FD
:10064A00A3E0F528A38006E4F527900001E0F52948
:10065A001528E529C378509640030207A0AB08AADB
:10066A0009A90A75F010E529A4F58285F083120C10
:10067A00CFFFE528D39F40028F287854E6B40109BA
:10068A007858E6F52CF52B8009E4F52B7819E61451
:10069A00F52C7858A62B7858E6D3952C40030207F8
:1006AA0094E4F526E526C395284003020789E5293F
:1006BA0075F010A4AB08250AF9E50935F0FA90009F
:1006CA0004120CCF30E203020784900001120CCF0F
:1006DA0064387041E528D394044011E5272526247F
:1006EA0002F582E43400F583E0FD80707852E6C3B7
:1006FA009526FFE49400FE74FE2FF58274FF3EF502
:10070A0083E0FDE52975F010A4AB08250AF9E5098F
:10071A0035F0FA8047AB08AA09A90A75F010E5294D
:10072A00A4F58285F083120CCFFF7852E6C39FFFAF
:10073A00E49400FE7C00EF2526FFEC3EFEEF252721
:10074A00FFEC3EFE74FF2FF58274FF3EF583E0FD59
:10075A00E52975F010A429F9EA35F0FA90000D128E
:10076A000EE07858E6FF18E68FF0A4FFE5262FF58D
:10077A0082E435F0F583ED120D0E05260206AEAFC2
:10078A002912288F7858060206A07858A62BE52544
:10079A00648870158010E529B4FF0E900002E0F518
:1007AA0020E525B488031226C3E52564A860030260
:1007BA0008EB7854E6B4010F7A007B327D01785851
:1007CA00E6FF1220C6801AE4F526E526C3781996B4
:1007DA00500F7A007B327D01AF261220C605268093
:1007EA00E9900001E030E711547FFEA3E0FDEEF549
:1007FA002DEDF52E752703800C900001E0752D0074
:10080A00F52E75270274002527F582E43400F58356
:10081A00E0FF74012527F582E43400F583E0F52A28
:10082A008F29E529D3952A40030208E8E529C378E8
:10083A00509640030208E3AB08AA09A90A75F0100A
:10084A00E529A4F58285F083120CCFF5287854E6C1
:10085A00B401097858E6F52CF52B8009E4F52B78D4
:10086A0019E614F52C7858A62B7858E6D3952C500F
:10087A005EE4F526E526C39528504AE52975F01069
:10088A00A4AB08250AF9E50935F0FA900004120C20
:10089A00CF20E22DE52725262402F582E43400F54F
:1008AA0083E0FD90000D120EE07858E6FF18E68FFF
:1008BA00F0A4FFE5262FF582E435F0F583ED120D5D
:1008CA000E052680AFAF2912288F785806809A78AD
:1008DA0058A62BE5282527F527052902082C1226D4
:0108EA00C34A
:0108EB0022EA
:10F000007880E664F1600302F60CE4F53FF54078A1
:04F0100081E6601F16
:0DF0140075450A75461300D546FCD545F636
:10F021000540E5407002053F64107004E53F642728
:10F0310070DCC2AF7584015398FC75FFDE75FFADBE
:10F04100E4F53BF53AE4F58420982EE4F53FF540EC
:0EF05100209822C3E5409488E53F94135017A1
:0DF05F0075450A75461300D546FCD545F6EB
:10F06C000540E54070DF053F80DBB28680CF859997
:10F07C003AC298E53A641A600302F14CF53FF54048
:0EF08C00209822C3E5409488E53F9413501766
:0DF09A0075450A75461300D546FCD545F6B0
:10F0A7000540E54070DF053F80DB30989285993B4E
:10F0B700C298E4F53FF540209822C3E5409488E5DF
:05F0C7003F94135017F7
:0DF0CC0075450A75461300D546FCD545F67E
:10F0D9000540E54070DF053F80DB20980302F046DC
:10F0E90085993BC298E4F53FF540209822C3E54055
:08F0F9009488E53F94135017C1
:0DF1010075450A75461300D546FCD545F648
:10F10E000540E54070DF053F80DB20980302F046A6
:09F11E0085993BC298C285C29993
:0DF1270075451475461300D546FCD545F618
:06F134007599783099FD89
:0DF13A0075450A75461300D546FCD545F60F
:10F14700D28502F5FEE53A6450600302F1DCF53F33
:10F15700F540209822C3E5409488E53F9413501763
:0DF1670075450A75461300D546FCD545F6E2
:10F174000540E54070DF053F80DB20980302F04640
:09F1840085993BC298C285C2992D
:0DF18D0075451475461300D546FCD545F6B2
:08F19A007599793099FDC299C5
:0DF1A20075451475461300D546FCD545F69D
:08F1AF007599013099FDC29928
:0DF1B70075451475461300D546FCD545F688
:06F1C400E4F5993099FD0D
:0DF1CA0075450A75461300D546FCD545F67F
:0FF1D700D28502F5FEE53A6401703EC285C29909
:0DF1E60075451475461300D546FCD545F659
:08F1F3007599783099FDC2996D
:0DF1FB0075451475461300D546FCD545F644
:06F20800E4F5993099FDC8
:0DF20E0075450A75461300D546FCD545F63A
:10F21B00D28502F5FEE53A6402600302F2E2F53FA5
:10F22B00F540209822C3E5409488E53F941350178E
:0DF23B0075450A75461300D546FCD545F60D
:10F248000540E54070DF053F80DB20980302F0466B
:10F2580085993BC298E4F53CE53B13B39286E53BC0
:10F2680025E0FEC3E49400EE94F0502AE53B7F00CD
:10F2780025E0FEC394E0501EE53B20E01FE4F58442
:10F2880043B701758F038E418F428F828E83F0536F
:10F29800B7F0F58F8003753CFFE4F584C285C29909
:0DF2A80075451475461300D546FCD545F696
:08F2B5007599783099FDC299AA
:0DF2BD0075451475461300D546FCD545F681
:06F2CA00853C993099FD1E
:0DF2D00075450A75461300D546FCD545F678
:10F2DD00D28502F5FEE53A6403600302F42DF53F95
:10F2ED00F540209822C3E5409488E53F94135017CC
:0DF2FD0075450A75461300D546FCD545F64B
:10F30A000540E54070DF053F80DB20980302F046A8
:10F31A0085993BC298E4F53FF540209822C3E54021
:08F32A009488E53F941350178D
:0DF3320075450A75461300D546FCD545F615
:10F33F000540E54070DF053F80DB20980302F04673
:10F34F0085993DC298E53B139286E53B25E0FEC3C8
:10F35F00E49400EE94F0400302F046E53B7D002577
:10F36F00E0FCC394E0400302F046E4F58443B701A8
:10F37F00758F01E53D75F020A42DFFE5F03CF541BB
:10F38F008F42E4F584F53EE53EC394205048E4F502
:10F39F003FF540209822C3E5409488E53F941350F1
:01F3AF001746
:0DF3B00075450A75461300D546FCD545F697
:10F3BD000540E54070DF053F80DB20980302F046F5
:10F3CD000542E542AE417002054114F5828E83E59A
:10F3DD0099F0C298053E80B1E4F58453B7F0F58FEE
:06F3ED00F584C285C299FF
:0DF3F30075451475461300D546FCD545F64A
:08F400007599783099FDC2995D
:0DF4080075451475461300D546FCD545F634
:06F41500E4F5993099FDB9
:0DF41B0075450A75461300D546FCD545F62B
:10F42800D28502F5FEE53A6404600302F4DDF53F97
:10F43800F540209822C3E5409488E53F941350177F
:0DF4480075450A75461300D546FCD545F6FE
:10F455000540E54070DF053F80DB20980302F0465C
:10F4650085993BC298E53B25E0F543754400E4F5F5
:10F475003CF53FF5400544E544AE437002054314B1
:10F48500F5828E83E493253CF53C0540E54070020A
:0EF49500053F7004E53F640270DBC285C2993A
:0DF4A30075451475461300D546FCD545F699
:08F4B0007599783099FDC299AD
:0DF4B80075451475461300D546FCD545F684
:06F4C500853C993099FD21
:0DF4CB0075450A75461300D546FCD545F67B
:10F4D800D28502F5FEE53A6405600302F5F3F53FCF
:10F4E800F540209822C3E5409488E53F94135017CF
:0DF4F80075450A75461300D546FCD545F64E
:10F505000540E54070DF053F80DB20980302F046AB
:10F5150085993BC298E4F53FF540209822C3E54024
:08F525009488E53F9413501790
:0DF52D0075450A75461300D546FCD545F618
:10F53A000540E54070DF053F80DB20980302F04676
:09F54A0085993DC298C285C29961
:0DF5530075451475461300D546FCD545F6E8
:08F5600075997F3099FDC299F5
:0DF5680075451475461300D546FCD545F6D3
:10F575007599203099FDE53B25E0FCE53D75F020CA
:10F58500A42400FFE5F03CF5438F44E4F53CF53E4B
:02F59500C29919
:0DF5970075451475461300D546FCD545F6A4
:10F5A400854482854383E493F5993099FD0544E5C8
:10F5B40044AE437002054314F5828E83E493253CE4
:0BF5C400F53C053EE53EB420C8C299AE
:0DF5CF0075451475461300D546FCD545F66C
:06F5DC00853C993099FD09
:0DF5E20075450A75461300D546FCD545F663
:10F5EF00D285800BE53AB40606E4F58475EF10E595
:0DF5FF003A6407600302F0467880F6D2AF50
:01F60C0022DB
:1022EA007F0012275320090B7A007B327D017F0081
:1022FA001220C6300C0B7A007B1E7D017F00122053
:10230A00C6300817300D147A007B327D017858E602
:10231A00FF1220C6C208121DB5D209200B0C300DBF
:10232A0009788076F1121DB5D20B300E08300D05F2
:10233A00C20E12F000200D1212000EE47B2C7A015C
:0B234A00F9F8C3120DFF5002D20D2263
:0B28840012109C1222EA12000380F8E0
:10197000005EBCE2613FDD83C29C7E20A3FD1F416F
:101980009DC3217FFCA2401E5F01E3BD3E6082DC5F
:10199000237D9FC1421CFEA0E1BF5D0380DE3C624F
:1019A000BEE0025CDF81633D7C22C09E1D43A1FF3F
:1019B0004618FAA427799BC584DA3866E5BB59072F
:1019C000DB856739BAE406581947A5FB7826C49A1F
:1019D000653BD987045AB8E6A7F91B45C6987A240F
:1019E000F8A6441A99C7257B3A6486D85B05E7B9FF
:1019F0008CD2306EEDB3510F4E10F2AC2F7193CDEF
:101A0000114FADF3702ECC92D38D6F31B2EC0E50DE
:101A1000AFF1134DCE90722C6D33D18F0C52B0EECE
:101A2000326C8ED0530DEFB1F0AE4C1291CF2D73BE
:101A3000CA947628ABF517490856B4EA6937D58BAE
:101A40005709EBB536688AD495CB2977F4AA48169E
:101A5000E9B7550B88D6346A2B7597C94A14F6A88E
:101A6000742AC896154BA9F7B6E80A54D7896B357E
:0A1A7000000000002B6096CBDDEEB5
:0328670001160A4D
:1021570015151515A815ECF608EDF6151515151531
:1021670015A815C6EBC608C6EAC608C6E9C6E5152A
:0421770024FCF5153A
:10217B00F80808E4F6A815F608F6E5152407F9A8FB
:10218B0015E6FE08E6FFC3099719E76480F8EE64CD
:10219B0080985037E5152404F8CBE6CB08E6FA080F
:1021AB00E6F98F828E83120CCFA815080866FFE51F
:1021BB00152403F8EFF6E690197093A8150808F6A6
:1021CB00A8150806E61870B20680AFA8150808E631
:0121DB00FF04
:0721DC00E5152409F51522A9
:0B287800ED6F7874F6E690197093FF86
:012883002232
:1027AA00EF7023F5847598D0F584759115F58475C5
:1027BA00C90875CBFFED901A6F93F5CA75C804E482
:0827CA00F584D2ACC2BCD2AF11
:0127D20022E4
:1023550090018D120E9500000000900191120E95CE
:10236500000000009001887464F0E47875F67875D3
:10237500E6FFC394015043EF25E025E02489F5826B
:10238500E43401F583E4F0EF25E025E0248AF582C5
:10239500E43401F583E4F0EF25E025E0248BF582B4
:1023A500E43401F583E4F0EF25E025E0248CF582A3
:0A23B500E43401F583E4F00680B47F
:0123BF0022FB
:1027F500D2AFD2A9C2BBE4F584E589540F4401F5F3
:0F28050089758E02758CAFE4F58AD28C0223554B
:021A7A00151540
:101A7C00A815E4F6A815E6FFC394014003021B6504
:101A8C00EF25E025E0248CF582E43401F583E0FFBA
:101A9C00D394005003021B21E625E025E0248AF5AF
:101AAC0082E43401F583E0706CEF30E019E6FF2539
:101ABC00E025E0248CF582E43401F583E0D3940135
:101ACC0040047D0080067D01A815E6FF122489A83C
:101ADC0015E6FF25E025E0248CF582E43401F5833E
:101AEC00E014F0EF25E025E0248CF582E43401F5D8
:101AFC0083E06021E6FF25E025E0248BF582E434C9
:101B0C0001F583E0FEEF25E025E0248AF582E4343C
:101B1C0001F583EEF0A815E6FF25E025E0248AF513
:101B2C0082E43401F583E06011EF25E025E0248A9E
:101B3C00F582E43401F583E014F0A815E6FF25E006
:101B4C0025E0248CF582E43401F583E070057D01F9
:091B5C00122489A81506021A8062
:031B650005152241
:03000B00021F963B
:101F9600C0E0C0F0C083C082C0D0E8C0E0E9C0E0C5
:101FA600EAC0E0EBC0E0ECC0E0EDC0E0EEC0E0EF80
:101FB600C0E0758CAF90018DE0FCA3E0FDA3E0FED0
:101FC600A3E02401FFE43EFEE43DFDE43CFC900179
:101FD6008D120E89900188E014F0E0702590019131
:101FE600E0FCA3E0FDA3E0FEA3E02401FFE43EFE47
:101FF600E43DFDE43CFC900191120E899001887449
:1020060064F0121A7A1227D3D0E0FFD0E0FED0E0B7
:10201600FDD0E0FCD0E0FBD0E0FAD0E0F9D0E0F86B
:0B202600D0D0D082D083D0F0D0E032C8
:102726001515A815EDF61515A815EFF6A815E6FF6B
:10273600C39401501308E6FEEF25E025E02489F551
:0D27460082E43401F583EEF005150515223F
:1020C60015151515A815EAF608EBF61515A815ED5C
:1020D600F61515A815EFF6A815E6FFC39401506A84
:1020E600EF25E025E0248CF582E43401F583E070E9
:1020F60059E6FB25E025E0248AF582E43401F583E0
:10210600E0704708E625E004FFA815E6FA25E02575
:10211600E0248CF582E43401F583EFF00808E6FE4E
:1021260008E6FF7C007D0A120D42EA25E025E02440
:102136008BF582E43401F583EFF0EB25E025E0240E
:102146008AF582E43401F583E4F0E5152404F515F7
:012156002266
:0E2489001515A815EDF61515A815EFF6151585
:10249700A81508E6FFC394015024EF25E025E024A2
:1024A70089F582E43401F583E06013A8150808E68E
:1024B70070047F0180027F00A8150808EFF6A815B1
:1024C700A68475840FA81508E67009A8150808E6FC
:0924D70024FF9286A815E6F584A5
:0724E0000515051505152285
:10000E00C2AF90018DE0FCA3E0FDA3E0FEA3E0FFF4
:02001E00D2AF5F
:0100200022BD
:10283300C2AF900191E0FCA3E0FDA3E0FEA3E0FFA3
:02284300D2AF12
:012845002270
:102753001515A815EFF6A815E670057817F608F60F
:10276300300F167816E675F064A4FFC37818E69F59
:0C27730018E695F0500375FFA50515222F
:10281400D20FE47817F608F6EF78166003F6800214
:0F282400760A75FF0775FFA5E4F58475EF0422AA
:10284600C20FE47817F608F6781676FF75FFDE7580
:03285600FFAD22B1
:1027D300781806E618700106300F167816E675F0BD
:1027E30064A4FFC37818E69F18E695F0500375FFBD
:0227F300A5221D
:04277F008E0D8F0E1E
:10278300E4F50FF510C3E510950EE50F950D501602
:102793007FE87E031224E77F011227530510E5101B
:0627A30070E3050F80DF6A
:0127A900220D
:0424E7008E118F12B1
:1024EB00D3E51294FAE5119400500EEFD39400400B
:1024FB00407E1600DEFD1F80F2851113851214D36A
:10250B00E51494FAE513940040157FFA7E0012242B
:10251B00E774062514F51474FF3513F51380E0D317
:10252B00E5129400E51194004007AF14AE1312248A
:01253B00E7B8
:01253C00227C
:1023C000754A00754B00754C447B007A0079427D5C
:0123D000020A
:0823D1008B468A4789488D49BB
:1023D9007F01122753AB4AAA4BA94C120D7824004E
:1023E900FFE5F034E0FE85464D85474E85484FE4CC
:1023F900FDEDC39549501BEF2DF582E43EF583E4CD
:1024090093AB4DAA4EA94F8D82758300120D0E0D07
:0F24190080DFAB4AAA4BA94CE48549F0020DA322
:101C5000753C12753D3475440075450075463E7BF4
:071C6000007A00793C7D02CF
:081C67008B408A4189428D4344
:101C6F007880E664F16003021D04122846C2AFE4D7
:101C7F00F58443B701758F01AB44AA45A946120DF0
:101C8F00782400FFE5F034E07875F608EFF6AA4106
:101C9F00A9427879A64008C6EAC608C6E9C6E4781C
:101CAF0077F67877E6C3954350327879CBE6CB0851
:101CBF000806E618CAE6CA70010614F9120CB678BF
:101CCF0078F6E6FF78750806E618CCE6CC700106C4
:101CDF0014F5828C83EFF078770680C6E4F58F5386
:101CEF00B7F0AB44AA45A9468543F0120DA3D2AF76
:051CFF00E4FF122814AF
:011D040022BC
:10262D007880E664F17046C2AF122846E4F5844323
:10263D00B701758F03787676E008F67875F67876BB
:10264D00E6FE08E6F5828E83E4F07F0112275378CB
:10265D0077E426F618740236F61806E6C394084099
:0D266D00DDE4F58F53B7F0D2AFFF12281453
:01267A00223D
:101DB50012262DE4F53EF53FF54475450075463E82
:101DC500FB7A00795A7D16121C67121C50E4F53B0C
:101DD500E53BC37819965073E4F53AAB08AA09A90F
:101DE5000A75F010E53AA4F58285F083120CCF60F0
:101DF50056E53A75F010A429F9EA35F0FA90000D88
:101E0500120EE07857E6853BF0A429F9EA35F0FA99
:101E1500EBC0E0EAC0E0E9C0E0AB08AA09A90A7591
:101E2500F010E53AA4F58285F083120CCFFD7544D8
:101E35000075450075463ED0E0F9D0E0FAD0E0FBEC
:101E4500121C67053A8094053B8085121C50E47886
:021E550080F615
:011E57002268
:021B68008F3EAE
:101B6A00E4F544F545F541F54A754B00754C44FBDF
:101B7A007A00795A7D161223D11223C0E5436434C0
:101B8A007004E54264127003434101E4F540E54004
:101B9A00C37819964003021C3BE4F53FAB08AA0937
:101BAA00A90A75F010E53FA4F58285F083120CCFDF
:101BBA00607AE53E6054E53F75F010A429F9EA35EC
:101BCA00F0FA90000D120EE07857E68540F0A4294D
:101BDA00F9EA35F0FAEBC0E0EAC0E0E9C0E0AB08A8
:101BEA00AA09A90A75F010E53FA4F58285F08312C7
:101BFA000CCFFD754A00754B00754C44D0E0F9D006
:101C0A00E0FAD0E0FB1223D1801DAB08AA09A90A89
:101C1A0075F010E53FA4F58285F083120CCF2545B7
:101C2A00F545E43544F544053F021BA60540021B71
:101C3A00981223C0E54364347004E54264127003C9
:051C4A00434102AF411F
:011C4F002272
:1008EC00020C6AE86480F8E933E83360110460F0C4
:1008FC00ED33EC337009E8FCE9FDEAFEEBFF220472
:10090C0060DED3EB9FEA9EE99DE8C2E78CF0C2F76C
:10091C0095F0400CE8CCF8E9CDF9EACEFAEBCFFB38
:10092C00120C3585D0F05804700320D5B3E8047050
:10093C00075002B2D5020C7492D5EC0460F7E4CCEB
:10094C00C0E0C398F8603B94186008400DD0E0FB01
:10095C00020C4CE4FBFAC9FC8028E830E406E4C93C
:10096C00FBE4CAFCE830E305E4C9CACBFCE8540755
:10097C006010F8C3E913F9EA13FAEB13FBEC13FC60
:10098C00D8F130F52FC3E49CFCEF9BFFEE9AFEED03
:10099C0099FDD0E0FBEF4E4D4C701222DB03020CA4
:1009AC0071EC2CFCEF33FFEE33FEED33FDED30E755
:1009BC00EB020C4CEF2BFFEE3AFEED39FDD0E0FBD9
:1009CC0050130BBB0003020C74ED13FDEE13FEEF82
:0809DC0013FFEC13FC020C4CAC
:1009E400EC4D6011E8497017ED33EC3304600DE40D
:1009F400FCFFFEFD22E933E8330470F8020C6A12AE
:100A04000C3558046009E4CC2481500628500902AE
:100A14000C74284003020C71C0E0EB4A7044B980A6
:100A240006D0E0FB020C60EF4E701CBD8008EBFFAB
:100A3400EAFEE9FD80EBE98DF0A4FEE5F0020ACDC3
:100A4400E9CDF9EAFEEBFFEF89F0A4FCE5F0CE89ED
:100A5400F0A42EFFE435F0CD89F0A42DFEE435F0AA
:100A64008067EF4E7005BD80D780C3EF8BF0A4ACD8
:100A7400F0EE8BF0A42CFCE435F0F8EF8AF0A42C13
:100A8400E5F038FCE433CB8DF0A42CFCE5F03BF826
:100A9400EE8AF0A42CFCE5F038F8E433CF89F0A416
:100AA4002CFCE5F038CF3400CE89F0A42FFFE5F01C
:100AB4003EFEE433C98DF0A42EFEE5F039CD8AF074
:100AC400A42FFFE5F03EFEE43DFD33D0E0FB5007EC
:100AD4000BBB000F020C74EC2CFCEF33FFEE33FE67
:060AE400ED33FD020C4C95
:100AEA00020C74EC5D046005E859047003020C6A98
:100AFA00120C35580460F6EC4860F2EC7004FDFE06
:100B0A00FF22C860DB2481C85009C39860025006DE
:100B1A00020C719850CAF582E9294B4A7005AB82DA
:100B2A00020C6075F0007C1A7880C3EF9BEE9AED98
:100B3A0099400DC3EF9BFFEE9AFEED99FDE842F056
:100B4A00DC23ACF0D0E0FFD0E0FED0E0FDAB8220A9
:100B5A00E7101BEB60BAEC2CFCEF33FFEE33FEED33
:100B6A0033FD020C4CE803F830E705C0F075F000DD
:100B7A00EF2FFFEE33FEED33FD40B830E7C280AA17
:100B8A0074F8CC6480CCC86480C8F582046043C31E
:100B9A00EB9FF5F0EA9E42F0E99D42F0E89C45F0B1
:100BAA0060305018E5825FFFE582F42B5582FB50D6
:100BBA00210ABA001D09B90019088016E5825BFBF3
:100BCA00E582F42F5582FF50090EBE00050DBD00C7
:100BDA00010CC3EB9FF5F0EA9E42F0E99D42F0E872
:0D0BEA009C45F06007CC4820E701B3EC22E9
:100BF70075F020800E75F010800575F0087D007E79
:100C0700007F003392D530D503120DDBEC33401053
:100C1700EF33FFEE33FEED33FDEC33FCD5F0ED2281
:0E0C2700E5F0247EA2D513CC92E7CDCEFF22BD
:101D05008F458E448D438C4274FFFFFEFDFCAB4531
:101D1500AA44A943A842C3120DFF602C7F807E967A
:101D25007D187C4BAB45AA44A943A842120B8A6097
:101D35000250157F807E967D187CCBAB45AA44A9C1
:101D450043A842120B8A5009AF45AE44AD43AC429D
:101D550022AF45AE44AD43AC42120C7F8F498E484D
:101D65008D478C46EC120BF7C8ECC8C9EDC9CAEE15
:101D7500CACBEFCBAF45AE44AD43AC421208EFE45E
:101D8500FBFAF9F8120B8A601A401874FF2549F519
:101D950049E54834FFF548E54734FFF547E546345E
:101DA500FFF546AF49AE48AD47AC46EC120BF722FE
:100C3500E9D2E7C933E833F892D5EDD2E7CD33EC05
:070C450033FC5002B2D5227E
:100C4C00EC30E7100FBF000C0EBE00080DBD000409
:100C5C000BEB6014A2D5EB13FCED92E7FD2274FFB5
:100C6C00FCFDFEFF22E480F8A2D574FF13FC7D800E
:030C7C00E480EF22
:100C7F00EDD2E7CD33EC3392D524814006E4FFFE6D
:100C8F00FDFC22FCE4CFCECDCC24E0501174FF80CC
:100C9F00EDC3CC13CCCD13CDCE13CECF13CF047069
:070CAF00F030D5DE020DDB81
:030000000221E3F7
:0C21E300787FE4F6D8FD75818102222A85
:100CB600BB010689828A83E0225002E722BBFE023C
:090CC600E32289828A83E493226F
:100CCF00BB010CE58229F582E5833AF583E02250DA
:100CDF0006E92582F8E622BBFE06E92582F8E22224
:0D0CEF00E58229F582E5833AF583E493223E
:100CFC00BB010689828A83F0225002F722BBFE01D7
:020D0C00F322D0
:100D0E00F8BB010DE58229F582E5833AF583E8F01B
:100D1E00225006E92582C8F622BBFE05E92582C8C7
:020D2E00F222AF
:100D3000EF8DF0A4A8F0CF8CF0A428CE8DF0A42ED7
:020D4000FE2291
:100D4200C2D5EC30E709B2D5E4C39DFDE49CFCEECC
:100D520030E715B2D5E4C39FFFE49EFE120F62C3D3
:100D6200E49DFDE49CFC8003120F6230D507C3E4CE
:060D72009FFFE49EFE223B
:100D7800BB010A89828A83E0F5F0A3E02250068746
:100D8800F009E71922BBFE07E3F5F009E319228908
:0B0D9800828A83E493F5F0740193223B
:100DA300BB010789828A83020FB7500B09C5F0275D
:100DB300F7C5F01937F722BBFE0D09F8E325F0F369
:100DC300C5F019E338F322F889828A8374019325E5
:080DD300F0C5F0F8E4933822AA
:0E0DDB00C3E49FFFE49EFEE49DFDE49CFC2229
:100DE900EB9FF5F0EA9E42F0E99D42F0EC6480C881
:060DF90064809845F02221
:100DFF00EB9FF5F0EA9E42F0E99D42F0E89C45F04A
:010E0F0022C0
:100E1000E8600FEFC333FFEE33FEED33FDEC33FC40
:030E2000D8F122E4
:100E2300BB010789828A83020FD95005E9F8020FB3
:100E3300CDBBFE05E9F8020FE589828A83020FF133
:100E4300BB010789828A83020E895005E9F8020EE5
:0A0E53007DBBFE05E9F8021037220E
:100E5D00BB010789828A8302100E5005E9F8021042
:100E6D0001BBFE05E9F802101A89828A8302102758
:0C0E7D00ECF608EDF608EEF608EFF622A1
:0C0E8900ECF0A3EDF0A3EEF0A3EFF022DC
:100E9500A8828583F0D083D082120EAC120EAC12DC
:100EA5000EAC120EACE473E493A3C583C5F0C58301
:100EB500C8C582C8F0A3C583C5F0C583C8C582C8A7
:010EC500220A
:100EC600BB010789828A83020E955005E9F8021054
:0A0ED60043BBFE05E9F802105C22A0
:100EE000BB010DE58229F582E5833AF58302107E88
:100EF0005007E92582F8021075BBFE07E92582F844
:100F0000021087E58229F582E5833AF58302109085
:100F1000D083D082F8E4937012740193700DA3A370
:100F200093F8740193F5828883E473740293686084
:060F3000EFA3A3A380DF84
:10253D008B3E8A3F8940E4F546F547E5451545AEA6
:10254D0044700215444E6033AB41AA42A943120CAC
:10255D00B6FFAB3EAA3FA9400547E547AC46700222
:10256D00054614F5828C83EF120D0EEF60CD7401CC
:10257D002543F543E43542F54280C0AB3EAA3FA961
:02258D004022EA
:100F3600EF4E6012EF60010EEDBB010B89828A83D2
:100F4600F0A3DFFCDEFA2289F05007F709DFFCA9DF
:0C0F5600F022BBFEFCF309DFFCA9F02236
:1021EF00022884E493A3F8E493A34003F68001F25A
:1021FF0008DFF48029E493A3F85407240CC8C333F1
:10220F00C4540F4420C8834004F456800146F6DFBF
:10221F00E4800B0102040810204080902859E47ECE
:10222F00019360BCA3FF543F30E509541FFEE493B4
:10223F00A360010ECF54C025E060A840B8E493A37B
:10224F00FAE493A3F8E493A3C8C582C8CAC583CAA6
:10225F00F0A3C8C582C8CAC583CADFE9DEE780BE5E
:01286A00006D
:100F6200BC000BBE0029EF8DF084FFADF022E4CC73
:100F7200F875F008EF2FFFEE33FEEC33FCEE9DEC3C
:100F8200984005FCEE9DFE0FD5F0E9E4CEFD22ED82
:100F9200F8F5F0EE8420D21CFEADF075F008EF2FCC
:100FA200FFED33FD4007985006D5F0F222C398FDBD
:050FB2000FD5F0EA225A
:100FB700C5F0F8A3E028F0C5F0F8E58215827002C5
:060FC7001583E038F02262
:0C0FCD00E6FC08E6FD08E6FE08E6FF2250
:0C0FD900E0FCA3E0FDA3E0FEA3E0FF228B
:0C0FE500E2FC08E2FD08E2FE08E2FF2248
:100FF100E493FC740193FD740293FE740393FF2246
:0D100100E6FB08E6F908E6FA08E6CBF8225F
:0C100E00E0F8A3E0F9A3E0FAA3E0FB2265
:0D101A00E2FB08E2F908E2FA08E2CBF82256
:10102700E493F8740193F9740293FA740393FB221F
:0C103700ECF208EDF208EEF208EFF222F5
:10104300D083D082E493F608740193F60874029374
:09105300F608740393F6740473AB
:10105C00D083D082E493F208740193F20874029363
:09106C00F208740393F27404739A
:09107500E6FB08E6FA08E6F922A0
:09107E00E0FBA3E0FAA3E0F92273
:09108700E2FB08E2FA08E2F9229A
:0C109000E493FB740193FA740293F922BC
:00000001FF
